:020000040000FA
:040000000DEF00F010
:0800080006EF20F0EBEF1EF003
:10001000FA6AFB6AD890E834F96E7AEC1FF016ECB5
:100020001FF00A0E29EC1FF00398BBEC1FF0030E23
:1000300009EC1FF0320E5FEC1FF0030E09EC1FF00D
:10004000320E5FEC1FF0030E09EC1FF0320E5FEC76
:100050001FF0320EF8EC1EF0280EF8EC1EF0969011
:100060009598969293909392939493969398939A4B
:10007000939C939E94809482948494869488948A8A
:10008000948C948E9580958295849586076A086AEB
:1000900000920094096A0A6A00860B6A0C6A0D6A6B
:1000A0000E6A0F6A106A116A126A9684959E959A72
:1000B000959C058EA1EC1FF0059AA5EC1FF0010E92
:1000C0004E6E010E4F6E0598A7EC1FF0B1EC11F0CB
:1000D00006809FEC1FF0D3EC1EF0D0EC1EF0500E0B
:1000E000EDEC1EF0720EEDEC1EF0650EEDEC1EF068
:1000F000610EEDEC1EF06D0EEDEC1EF0700EEDECF1
:100100001EF0200EEDEC1EF0560EEDEC1EF0650E0E
:10011000EDEC1EF0720EEDEC1EF02E0EEDEC1EF06E
:10012000200EEDEC1EF0310EEDEC1EF02E0EEDEC7F
:100130001EF0310EEDEC1EF0300EEDEC1EF0CDECAD
:100140001EF0200EEDEC1EF0200EEDEC1EF0450E24
:10015000EDEC1EF06C0EEDEC1EF0650EEDEC1EF0FD
:100160006B0EEDEC1EF0740EEDEC1EF06F0EEDEC70
:100170001EF0720EEDEC1EF0200EEDEC1EF0320EB5
:10018000EDEC1EF0300EEDEC1EF0300EEDEC1EF03E
:10019000340EEDEC1EF0200EEDEC1EF0200EEDEC1A
:1001A0001EF00A0ECCEC15F0D3EC1EF0506A92EC67
:1001B0001FF05150136E13502A08D8B4E4EF00F02A
:1001C000B9EC12F03BEC13F061EC14F082A0F2EF0A
:1001D00000F0C7EC02F061EC14F031EC11F01650B5
:1001E00036EC11F04B500108D8A4FBEF00F0146A74
:1001F000156A31EC11F04B500208D8A41AEF01F047
:10020000D3EC1EF0CDEC1EF013EC1AF0CAEC1EF08D
:10021000BEEC1EF07CEC12F0C9EC11F00952D8A42F
:1002200018EF01F07CEC12F0C9EC11F00EEF01F0C8
:10023000D3EC1EF04B500308D8A425EF01F04C502E
:10024000146E4D50156E31EC11F0165036EC11F065
:100250000588A7EC1FF026500108D8A440EF01F054
:1002600024EC1DF0CAEC1EF0A6EC1EF015500D6E2D
:1002700014500C6E156A146ADDEC10F042EF01F0B8
:1002800031EC11F0010E0B6E010E0F6E008600A610
:1002900077EF01F0C8EC0EF027EC13F00096010E9A
:1002A0000B6E010E0F6E24500108D8B45DEF01F003
:1002B00024500208D8A462EF01F006929DEC1FF0D2
:1002C00065EF01F006829DEC1FF025500108D8B4BF
:1002D0006FEF01F025500208D8A474EF01F00680FA
:1002E0009FEC1FF077EF01F006909FEC1FF00F508E
:1002F0005B6E640E5C6EF3EC1FF0506E50500108A4
:10030000D8A493EF01F024500208D8A48BEF01F099
:1003100006829DEC1FF025500208D8A493EF01F04F
:1003200006909FEC1FF00B500001FF08D8A49FEF30
:1003300001F0C8EC0EF0010E0B6E116A126A7CEC33
:1003400012F0C9EC11F009500C08D8A4C6EF01F066
:100350000598A7EC1FF0D3EC1EF0CDEC1EF0BEEC20
:100360001EF0050E21EC1FF07CEC12F0C9EC11F030
:100370000952D8A4C2EF01F07CEC12F0C9EC11F0E4
:10038000B8EF01F00588A7EC1FF0008609500808B7
:10039000D8B4D2EF01F009500408D8B4D2EF01F07C
:1003A000126A116A09500808D8A4EAEF01F099EC22
:1003B0000DF0122A116A12500A08D8B0EAEF01F0C3
:1003C00099EC0DF099EC0DF099EC0DF099EC0DF025
:1003D00099EC0DF009500408D8A402EF02F0ADEC3E
:1003E0000DF0112A126A11500A08D8B002EF02F07B
:1003F000ADEC0DF0ADEC0DF0ADEC0DF0ADEC0DF0A5
:10040000ADEC0DF009500308D8A41CEF02F0D89011
:100410001530516ED89014305124146E1450156E4E
:1004200031EC11F009500308D8A41BEF02F07CEC6A
:1004300012F012EF02F0008614500008D8B032EF2C
:1004400002F01750155CD8B032EF02F009500108E5
:10045000D8A432EF02F0010E145C146E152A31ECB0
:1004600011F000861750145CD8B048EF02F0155018
:100470000008D8B048EF02F009500208D8A448EFAD
:1004800002F0142A010E155C156E31EC11F0008695
:100490000A500108D8A453EF02F081B053EF02F0E4
:1004A000010EBDEC0DF00A500208D8A45EEF02F078
:1004B00081B25EEF02F0020EBDEC0DF00A500408AE
:1004C000D8A469EF02F081B469EF02F0030EBDEC2D
:1004D0000DF00A500808D8A474EF02F081B674EF4A
:1004E00002F0040EBDEC0DF081B883EF02F028524B
:1004F000D8A483EF02F00A501008D8A483EF02F0CA
:10050000050EBDEC0DF081BA92EF02F02852D8A48E
:1005100092EF02F00A502008D8A492EF02F0060EE3
:10052000BDEC0DF081BCA1EF02F02852D8A4A1EFE0
:1005300002F00A504008D8A4A1EF02F0070EBDEC6B
:100540000DF081BEB1EF02F02852D8A4B1EF02F055
:100550000A5000018008D8A4B1EF02F0080EBDECEB
:100560000DF00B2A0F2A1450175CD8A0BDEF02F033
:100570001550175CD8B0C3EF02F01750146E175027
:10058000156E31EC11F047EF01F0C5EF02F0D3EC3E
:100590001EF0D0EC1EF0530EEDEC1EF0650EEDECEF
:1005A0001EF0740EEDEC1EF0750EEDEC1EF0700EEC
:1005B000EDEC1EF0200EEDEC1EF0200EEDEC1EF02A
:1005C000560EEDEC1EF0650EEDEC1EF0720EEDEC2D
:1005D0001EF02E0EEDEC1EF0200EEDEC1EF0310E96
:1005E000EDEC1EF02E0EEDEC1EF0300EEDEC1EF0DC
:1005F000300EEDEC1EF00A0ECCEC15F0D3EC1EF034
:10060000020E2EEC03F07CEC12F009500408D8A482
:100610000DEF03F0010E2EEC03F009500808D8A4EA
:1006200015EF03F0000E2EEC03F009500208D8A4D9
:100630001EEF03F03BEC13F02DEF03F0095001081F
:10064000D8A42BEF03F0ABEC03F0050E21EC1FF068
:10065000020E2EEC03F003EF03F01200506E505028
:100660000108D8A435EF03F04F2A5052D8A43CEF2C
:1006700003F0010E4F5C4F6E4F52D8A442EF03F0CF
:100680000D0E4F6E4F500D08D8B049EF03F0010E1C
:100690004F6ED3EC1EF04F500108D8A452EF03F078
:1006A000C1EC1DF04F500208D8A459EF03F0A1ECA3
:1006B0001DF04F500308D8A460EF03F077EC1DF055
:1006C0004F500408D8A467EF03F0F7EC1CF04F502C
:1006D0000508D8A46EEF03F0D9EC1CF04F500608C3
:1006E000D8A475EF03F08CEC1CF04F500708D8A489
:1006F0007CEF03F069EC1CF04F500808D8A483EF9E
:1007000003F066EC1DF04F500908D8A48AEF03F0FF
:100710003CEC1DF04F500A08D8A491EF03F0DDEC3B
:100720001DF04F500B08D8A498EF03F0D7EC1DF044
:100730004F500C08D8A49FEF03F0FBEC19F04F507A
:100740000D08D8A4A6EF03F0AAEC1CF042EC1CF0B4
:10075000030E21EF1FF04F500108D8A4B5EF03F0AE
:1007600082EC0AF0030E21EC1FF04F500208D8A4CF
:10077000BFEF03F007EC0AF0030E21EC1FF04F501F
:100780000308D8A4C9EF03F0CCEC09F0030E21EC68
:100790001FF04F500408D8A4D3EF03F036EC07F055
:1007A000030E21EC1FF04F500508D8A4DAEF03F038
:1007B000C1EC0CF04F500608D8A4E4EF03F088EC2D
:1007C00009F0030E21EC1FF04F500708D8A4EEEFFC
:1007D00003F009EC08F0030E21EC1FF04F5008085D
:1007E000D8A4F8EF03F0C0EC04F0030E21EC1FF0E6
:1007F0004F500908D8A402EF04F0D9EC06F0030E1C
:1008000021EC1FF04F500A08D8A40CEF04F084EC40
:1008100006F0030E21EC1FF04F500B08D8A416EF82
:1008200004F02FEC06F0030E21EC1FF04F500C08E3
:10083000D8A420EF04F02AEC04F0030E21EC1FF002
:100840004F500D08D8A429EF04F0B9EC12F029EFAD
:1008500004F01200020E506E505087EC04F07CEC55
:1008600012F009500108D8A444EF04F050500108D8
:10087000D8A43FEF04F0020E506E41EF04F0010ED9
:10088000506E505087EC04F009500408D8A45EEF75
:1008900004F050500108D8A457EF04F04B2A4B50F5
:1008A0000408D8A455EF04F04B6A5BEF04F0145031
:1008B0004C6E15504D6E505087EC04F009500808EE
:1008C000D8A47AEF04F050500108D8A473EF04F0D4
:1008D0004B52D8A46EEF04F0040E4B6E010E4B5C2D
:1008E0004B6E77EF04F014504C6E15504D6E505017
:1008F00087EC04F0030E21EC1FF009500208D8A485
:1009000084EF04F086EF04F02FEF04F01200516E34
:10091000D3EC1EF051500108D8A4BAEF04F04B52AA
:10092000D8A495EF04F05EEC1EF04B500108D8A45B
:100930009CEF04F0BEEC1EF04B500208D8A4B1EFBF
:1009400004F0BEEC1EF0200EEDEC1EF02D0EEDECD2
:100950001EF03E0EEDEC1EF0200EEDEC1EF05EECF7
:100960001EF04B500308D8A4B8EF04F001EC1AF0C5
:10097000BCEF04F0CBEC19F0CDEC1EF028EF1CF02E
:10098000010E506E50500108D8A4E4EF04F0D3ECEF
:100990001EF0430EEDEC1EF0680EEDEC1EF04E5016
:1009A000300FEDEC1EF03A0EEDEC1EF0200EEDECEB
:1009B0001EF04E50EDEC05F0DFEC0FF028EC1CF0D3
:1009C000506A030E21EC1FF07CEC12F00950040871
:1009D000D8A455EF05F04E500108D8A4F8EF04F064
:1009E000312A31502408D8B0F8EF04F0010E316EEE
:1009F0004E500208D8A405EF05F0322A32502408E0
:100A0000D8B005EF05F0010E326E4E500308D8A4A1
:100A100012EF05F0332A33502408D8B012EF05F056
:100A2000010E336E4E500408D8A41FEF05F0342A8F
:100A300034502408D8B01FEF05F0010E346E4E502C
:100A40000508D8A42CEF05F0352A35502408D8B075
:100A50002CEF05F0010E356E4E500608D8A439EF84
:100A600005F0362A36502408D8B039EF05F0010ECB
:100A7000366E4E500708D8A446EF05F0372A375097
:100A80002408D8B046EF05F0010E376E4E50080826
:100A9000D8A453EF05F0382A38502408D8B053EFC3
:100AA00005F0010E386E010E506E09500808D8A4EA
:100AB000D4EF05F04E500108D8A469EF05F031508D
:100AC0000108D8A466EF05F0250E316E010E315CE9
:100AD000316E4E500208D8A478EF05F0325001086C
:100AE000D8A475EF05F0250E326E010E325C326E21
:100AF0004E500308D8A487EF05F033500108D8A45E
:100B000084EF05F0250E336E010E335C336E4E50CC
:100B10000408D8A496EF05F034500108D8A493EF48
:100B200005F0250E346E010E345C346E4E5005080F
:100B3000D8A4A5EF05F035500108D8A4A2EF05F020
:100B4000250E356E010E355C356E4E500608D8A464
:100B5000B4EF05F036500108D8A4B1EF05F0250E2A
:100B6000366E010E365C366E4E500708D8A4C3EFC1
:100B700005F037500108D8A4C0EF05F0250E376EF8
:100B8000010E375C376E4E500808D8A4D2EF05F03E
:100B900038500108D8A4CFEF05F0250E386E010EAD
:100BA000385C386E010E506E09500108D8A4E3EF8E
:100BB00005F04E2A4E500908D8A4E1EF05F0010EC9
:100BC0004E6E010E506E09500208D8A4EAEF05F0EF
:100BD000ECEF05F0C2EF04F01200526E5250010823
:100BE000D8A4F6EF05F031502EEF06F0525002086F
:100BF000D8A4FEEF05F032502EEF06F05250030855
:100C0000D8A406EF06F033502EEF06F05250040839
:100C1000D8A40EEF06F034502EEF06F0525005081F
:100C2000D8A416EF06F035502EEF06F05250060805
:100C3000D8A41EEF06F036502EEF06F052500708EB
:100C4000D8A426EF06F037502EEF06F052500808D1
:100C5000D8A42EEF06F038502EEF06F012005EEC0E
:100C600006F07CEC12F009500408D8A441EF06F01D
:100C7000252A25500308D8A43FEF06F0256A5EEC2C
:100C800006F009500808D8A451EF06F02552D8A460
:100C90004CEF06F0030E256E010E255C256E5EEC12
:100CA00006F0020E21EC1FF009500208D8A45BEFF9
:100CB00006F05DEF06F031EF06F01200D3EC1EF007
:100CC00025500108D8A46DEF06F019EC1EF0CAEC0F
:100CD0001EF08BEC1EF080EF06F025500208D8A421
:100CE0007AEF06F040EC1EF0CAEC1EF082EC1EF02B
:100CF00080EF06F019EC1EF0CAEC1EF082EC1EF03C
:100D0000CDEC1EF022EF1CF0B3EC06F07CEC12F000
:100D100009500408D8A496EF06F0242A24500308AA
:100D2000D8A494EF06F0246AB3EC06F00950080842
:100D3000D8A4A6EF06F02452D8A4A1EF06F0030E23
:100D4000246E010E245C246EB3EC06F0020E21EC3E
:100D50001FF009500208D8A4B0EF06F0B2EF06F079
:100D600086EF06F01200D3EC1EF024500108D8A440
:100D7000C2EF06F019EC1EF0CAEC1EF08BEC1EF070
:100D8000D5EF06F024500208D8A4CFEF06F040ECCF
:100D90001EF0CAEC1EF082EC1EF0D5EF06F019EC46
:100DA0001EF0CAEC1EF082EC1EF0CDEC1EF022EF1D
:100DB0001CF0010E506E50500108D8A408EF07F047
:100DC000D3EC1EF0480EEDEC1EF0570EEDEC1EF0CD
:100DD0003A0EEDEC1EF0200EEDEC1EF03952D8A4C8
:100DE000F4EF06F088EC1AF039500108D8A4FBEFB4
:100DF00006F06AEC1AF039500208D8A402EF07F0A6
:100E000049EC1AF022EC1CF0506A030E21EC1FF0A2
:100E10007CEC12F009500408D8A41AEF07F03950FE
:100E20000208D8A417EF07F0396A18EF07F0392A3B
:100E3000010E506E09500808D8A42CEF07F0395263
:100E4000D8A427EF07F0020E396E2AEF07F0010E43
:100E5000395C396E010E506E09500208D8A433EF88
:100E600007F035EF07F0DBEF06F01200010E506ED1
:100E7000008800A85DEF07F0D3EC1EF05050010889
:100E8000D8A44BEF07F0F9EC1CF0AFEC07F097ECAF
:100E90001EF058EF07F010EC1DF026500108D8A402
:100EA00056EF07F00AEC1EF058EF07F004EC1EF0C6
:100EB000CDEC1EF028EC1CF000987CEC12F00950F0
:100EC0000108D8A472EF07F0008850500108D8A498
:100ED0006DEF07F0506A6FEF07F0010E506E030ED2
:100EE00021EC1FF009500408D8B47CEF07F009503A
:100EF0000808D8A4A5EF07F05052D8A48CEF07F04B
:100F00002652D8A488EF07F0010E266E89EF07F06D
:100F1000266A0088A2EF07F009500408D8A499EFC8
:100F200007F0FF0E275CD8B097EF07F0272AA1EF54
:100F300007F027500108D8B0A1EF07F0010E275C99
:100F4000276E0088020E21EC1FF009500208D8A479
:100F5000ACEF07F0AEEF07F039EF07F01200008AB0
:100F60002750516E51505B6E640E5C6EF3EC1FF0B7
:100F7000526E52500008D8A4C3EF07F0200EEDECDB
:100F80001EF0CFEF07F051505B6E640E5C6EF3EC19
:100F90001FF0536E5350300FEDEC1EF0009A51507D
:100FA000586E640E596EE2EC1FF0536E5350516E42
:100FB00051505B6E0A0E5C6EF3EC1FF0546E545091
:100FC0000008D8A4F1EF07F000AAECEF07F0200E1C
:100FD000EDEC1EF0EFEF07F0300EEDEC1EF0FCEF45
:100FE00007F051505B6E0A0E5C6EF3EC1FF0556E0D
:100FF0005550300FEDEC1EF05150586E0A0E596EE0
:10100000E2EC1FF0556E5550516E5150300FEDEF20
:101010001EF0080E506ED3EC1EF0505056EC1CF033
:10102000505025EC09F013EC1EF028EC1CF07CEC81
:1010300012F009500408D8A42CEF08F05050CBEC63
:1010400008F0D0EC1EF0505056EC1CF0505025EC3F
:1010500009F0030E21EC1FF009500808D8A43FEF57
:1010600008F0505061EC08F0D0EC1EF0505056ECF7
:101070001CF0505025EC09F0030E21EC1FF0095034
:101080000208D8A446EF08F060EF08F00950010804
:10109000D8A45EEF08F0502A50500908D8A453EFA6
:1010A00008F0010E506ED0EC1EF0505056EC1CF0C3
:1010B000505025EC09F0030E21EC1FF017EF08F05B
:1010C0001200516E51500108D8A46FEF08F029505A
:1010D0000008D8B06FEF08F0010E295C296E51505E
:1010E0000208D8A47CEF08F02A500008D8B07CEFA2
:1010F00008F0010E2A5C2A6E51500308D8A489EF2B
:1011000008F02B500008D8B089EF08F0010E2B5CD6
:101110002B6E51500408D8A496EF08F02C5000080C
:10112000D8B096EF08F0010E2C5C2C6E51500508DB
:10113000D8A4A3EF08F02D500008D8B0A3EF08F012
:10114000010E2D5C2D6E51500608D8A4B0EF08F0AA
:101150002E500008D8B0B0EF08F0010E2E5C2E6EB5
:1011600051500708D8A4BDEF08F02F500008D8B0A0
:10117000BDEF08F0010E2F5C2F6E51500808D8A467
:10118000CAEF08F030500008D8B0CAEF08F0010EDE
:10119000305C306E1200516E51500108D8A4D7EF68
:1011A00008F0FF0E295CD8B0D7EF08F0292A51507B
:1011B0000208D8A4E2EF08F0FF0E2A5CD8B0E2EFF4
:1011C00008F02A2A51500308D8A4EDEF08F0FF0ECA
:1011D0002B5CD8B0EDEF08F02B2A51500408D8A4AE
:1011E000F8EF08F0FF0E2C5CD8B0F8EF08F02C2ACE
:1011F00051500508D8A403EF09F0FF0E2D5CD8B0BC
:1012000003EF09F02D2A51500608D8A40EEF09F07B
:10121000FF0E2E5CD8B00EEF09F02E2A51500708B1
:10122000D8A419EF09F0FF0E2F5CD8B019EF09F020
:101230002F2A51500808D8A424EF09F0FF0E305C83
:10124000D8B024EF09F0302A1200516E5150010835
:10125000D8A42FEF09F02950526E6CEF09F05150CD
:101260000208D8A438EF09F02A50526E6CEF09F04A
:1012700051500308D8A441EF09F02B50526E6CEF87
:1012800009F051500408D8A44AEF09F02C50526ECE
:101290006CEF09F051500508D8A453EF09F02D5018
:1012A000526E6CEF09F051500608D8A45CEF09F0BB
:1012B0002E50526E6CEF09F051500708D8A465EF1C
:1012C00009F02F50526E6CEF09F051500808D8A465
:1012D0006CEF09F03050526E525000018008D8A4D3
:1012E00076EF09F0C00E526E85EF09F0800E525C69
:1012F000D8B081EF09F052508008C008526E85EFD7
:1013000009F0800E525CC00F526E525048EF0FF041
:10131000D3EC1EF022EC1CF02852D8A494EF09F074
:10132000DCEC1BF096EF09F0B7EC1BF07CEC12F054
:1013300009500408D8A4ADEF09F02852D8A4A7EFAB
:1013400009F0010E286EB7EC1BF0AAEF09F0286A2D
:10135000DCEC1BF0030E21EC1FF009500808D8A4A8
:10136000C2EF09F02852D8A4BCEF09F0010E286E94
:10137000B7EC1BF0BFEF09F0286ADCEC1BF0030EA2
:1013800021EC1FF009500208D8A4C9EF09F0CBEFF7
:1013900009F096EF09F01200010E506E00887CEC07
:1013A00012F000A8E0EF09F0D3EC1EF028EC1AF0E0
:1013B000175048EC0FF0CDEC1EF022EC1CF000981A
:1013C00009500408D8A4ECEF09F0FF0E175CD8B060
:1013D000ECEF09F0172A008809500808D8A4FAEFA2
:1013E00009F017500108D8B0FAEF09F0010E175CA8
:1013F000176E0088020E21EC1FF009500208D8A4D5
:1014000004EF0AF006EF0AF0CFEF09F012002FEC1C
:1014100017F05250506E5350516E009800BC008827
:10142000009A00BE008AD3EC1EF0D0EC1EF0610ED4
:10143000EDEC1EF03A0EEDEC1EF0200EEDEC1EF081
:10144000040E536E5050546E200E32EC0DF0200EF0
:10145000EDEC1EF02F0EEDEC1EF0200EEDEC1EF06C
:10146000630EEDEC1EF03A0EEDEC1EF0200EEDECEE
:101470001EF0040E536E5150546E200E32EC0DF0DF
:10148000CDEC1EF0740EEDEC1EF03A0EEDEC1EF0FD
:10149000200EEDEC1EF000A853EF0AF0310EEDEC3B
:1014A0001EF056EF0AF0300EEDEC1EF0200EEDECC3
:1014B0001EF06F0EEDEC1EF06B0EEDEC1EF03A0E12
:1014C000EDEC1EF0200EEDEC1EF000AA6DEF0AF020
:1014D000310EEDEC1EF070EF0AF0300EEDEC1EF068
:1014E000200EEDEC1EF0140ECCEC15F07CEC12F09E
:1014F00009500208D8A47FEF0AF081EF0AF007EF45
:101500000AF01200010E506E010E516E030E21EC16
:101510001FF02FEC17F05250076E5350086E0092D8
:1015200000BC0082009400BE008400A49DEF0AF07D
:101530005150C4EC0AF0010E506E50500108D8A46E
:10154000A6EF0AF051503BEC0BF0506A7CEC12F025
:1015500009500208D8A4AFEF0AF0C3EF0AF009500F
:101560000108D8A4BEEF0AF0512A51500E08D8A4A1
:10157000BCEF0AF0010E516E010E506E030E21EC0D
:101580001FF089EF0AF01200526E52500108D8A4E1
:10159000CEEF0AF007503B6E08503C6E52500208E6
:1015A000D8A4D7EF0AF007503D6E08503E6E525057
:1015B0000308D8A4E0EF0AF007503F6E0850406ED1
:1015C00052500408D8A4E9EF0AF00750416E0850C1
:1015D000426E52500508D8A4F2EF0AF00750436E4D
:1015E0000850446E52500608D8A4FBEF0AF007508A
:1015F000456E0850466E52500708D8A404EF0BF011
:101600000750476E0850486E52500808D8A40DEF96
:101610000BF00750496E08504A6E52500908D8A482
:1016200016EF0BF007501B6E08501C6E52500A0844
:10163000D8A41FEF0BF00750196E08501A6E5250C5
:101640000B08D8A428EF0BF007501D6E08501E6E33
:1016500052500C08D8A431EF0BF007501F6E085001
:10166000206E52500D08D8A43AEF0BF00750216EAF
:101670000850226E1200526ED3EC1EF05250010838
:10168000D8A45DEF0BF091EC1EF05250300FEDEC52
:101690001EF0CAEC1EF0B2EC1EF0040E536E3B506E
:1016A000546E200E32EC0DF09DEC1EF0040E536EC5
:1016B0003C50546E200E32EC0DF052500208D8A46B
:1016C0007CEF0BF091EC1EF05250300FEDEC1EF061
:1016D000CAEC1EF0B2EC1EF0040E536E3D50546E78
:1016E000200E32EC0DF09DEC1EF0040E536E3E50B9
:1016F000546E200E32EC0DF052500308D8A49BEF2C
:101700000BF091EC1EF05250300FEDEC1EF0CAECD5
:101710001EF0B2EC1EF0040E536E3F50546E200EBD
:1017200032EC0DF09DEC1EF0040E536E4050546EE2
:10173000200E32EC0DF052500408D8A4BAEF0BF092
:1017400091EC1EF05250300FEDEC1EF0CAEC1EF082
:10175000B2EC1EF0040E536E4150546E200E32EC6B
:101760000DF09DEC1EF0040E536E4250546E200E90
:1017700032EC0DF052500508D8A4D9EF0BF091ECE3
:101780001EF05250300FEDEC1EF0CAEC1EF0B2EC21
:101790001EF0040E536E4350546E200E32EC0DF0CA
:1017A0009DEC1EF0040E536E4450546E200E32EC2D
:1017B0000DF052500608D8A4F8EF0BF091EC1EF093
:1017C0005250300FEDEC1EF0CAEC1EF0B2EC1EF0E1
:1017D000040E536E4550546E200E32EC0DF09DEC0D
:1017E0001EF0040E536E4650546E200E32EC0DF077
:1017F00052500708D8A417EF0CF091EC1EF052508D
:10180000300FEDEC1EF0CAEC1EF0B2EC1EF0040E30
:10181000536E4750546E200E32EC0DF09DEC1EF0CE
:10182000040E536E4850546E200E32EC0DF05250A0
:101830000808D8A436EF0CF091EC1EF05250300F8F
:10184000EDEC1EF0CAEC1EF0B2EC1EF0040E536E6E
:101850004950546E200E32EC0DF09DEC1EF0040E3B
:10186000536E4A50546E200E32EC0DF0525009085F
:10187000D8A451EF0CF076EC1EF0CAEC1EF0B2ECDE
:101880001EF0040E536E1B50546E200E32EC0DF001
:101890009DEC1EF0040E536E1C50546E200E32EC64
:1018A0000DF052500A08D8A46CEF0CF0A6EC1EF014
:1018B000CAEC1EF0B2EC1EF0040E536E1950546EBA
:1018C000200E32EC0DF09DEC1EF0040E536E1A50FB
:1018D000546E200E32EC0DF052500B08D8A487EF56
:1018E0000CF06AEC1EF0CAEC1EF0B2EC1EF0040E16
:1018F000536E1D50546E200E32EC0DF09DEC1EF018
:10190000040E536E1E50546E200E32EC0DF05250E9
:101910000C08D8A4A2EF0CF04FEC1EF0CAEC1EF09D
:10192000B2EC1EF0040E536E1F50546E200E32ECBB
:101930000DF09DEC1EF0040E536E2050546E200EE0
:1019400032EC0DF052500D08D8A4BDEF0CF0BEECF7
:101950001EF0CAEC1EF0B2EC1EF0040E536E2150C5
:10196000546E200E32EC0DF09DEC1EF0040E536E02
:101970002250546E200E32EC0DF0CDEC1EF028EF0C
:101980001CF0D3EC1EF0D9EC1CF0050E506EB1EC3F
:1019900011F0030E21EC1FF00480B7EC1FF004825D
:1019A000B5EC1FF00484B3EC1FF00486B1EC1FF01B
:1019B0000488AFEC1FF0048AADEC1FF0048CABEC94
:1019C0001FF0048EA9EC1FF0030E21EC1FF0502E27
:1019D000C7EF0CF0B1EC11F0030E506E0480B7ECC1
:1019E0001FF0030E21EC1FF0B1EC11F00482B5ECF6
:1019F0001FF0030E21EC1FF0B1EC11F00484B3ECE6
:101A00001FF0030E21EC1FF0B1EC11F00486B1ECD5
:101A10001FF0030E21EC1FF0B1EC11F00488AFECC5
:101A20001FF0030E21EC1FF0B1EC11F0048AADECB5
:101A30001FF0030E21EC1FF0B1EC11F0048CABECA5
:101A40001FF0030E21EC1FF0B1EC11F0048EA9EC95
:101A50001FF0030E21EC1FF0B1EC11F0502EEEEF51
:101A60000CF01200556E5350586E54505B6E640E5D
:101A70005C6EF3EC1FF0596E5950596E55506FEC77
:101A80000DF05A50556E5450586E640E596EE2EC7B
:101A90001FF0566E5650546E5350586E54505B6E35
:101AA0000A0E5C6EF3EC1FF05A6E5A50596E555088
:101AB0006FEC0DF05A50556E5450586E0A0E596E18
:101AC000E2EC1FF0576E5750546E5350586E5450FE
:101AD000596E55506FEC0DF05A50556E12005A6EFB
:101AE0005952D8A480EF0DF05A52D8B47EEF0DF0C1
:101AF0005A50026E020E582408EC00F098EF0DF0D8
:101B00000A0E595CD8B08EEF0DF05950300F026EAE
:101B1000020E582408EC00F096EF0DF00A0E595C06
:101B2000410F026E020E582408EC00F0300E5A6E7F
:101B3000120014500008D8B0ACEF0DF0155000089A
:101B4000D8B0ACEF0DF0010E145C146E010E155CF4
:101B5000156E31EC11F0008612001750145CD8B0ED
:101B6000BCEF0DF01750155CD8B0BCEF0DF0142A87
:101B7000152A31EC11F000861200526E010E0F6E24
:101B800024500008D8B0C8EF0DF006809FEC1FF07D
:101B900000865250166E26500108D8A4E1EF0DF0D1
:101BA00027500008D8B0E1EF0DF003EC11F05250CF
:101BB000F6EC0DF0525036EC11F0DDEC10F0F5EFD4
:101BC0000DF00598A7EC1FF0010E21EC1FF052500C
:101BD000F6EC0DF0525036EC11F031EC11F0010E34
:101BE00021EC1FF00588A7EC1FF01200536E535034
:101BF0000108D8A4FEEF0DF02950546E535002088E
:101C0000D8A405EF0EF02A50546E53500308D8A400
:101C10000CEF0EF02B50546E53500408D8A413EF61
:101C20000EF02C50546E53500508D8A41AEF0EF045
:101C30002D50546E53500608D8A421EF0EF02E50AC
:101C4000546E53500708D8A428EF0EF02F50546E4E
:101C500053500808D8A42FEF0EF03050546E26527F
:101C6000D8A437EF0EF014500C6E15500D6E0C50BA
:101C7000175C566E0D50175C576E800E185CD8B00E
:101C80005BEF0EF018508008556E5650555CD8B07A
:101C90005BEF0EF05750555CD8B05BEF0EF026525C
:101CA000D8A457EF0EF05550142655501526555010
:101CB0000C2655500D26185000018008D8B07EEF34
:101CC0000EF0800E185C556E0C50555CD8B07EEF4F
:101CD0000EF00D50555CD8B07EEF0EF02652D8A411
:101CE00078EF0EF05550145C146E5550155C156E5F
:101CF00055500C5C0C6E55500D5C0D6E5450186EAA
:101D00000C50175C566E0D50175C576E1850000142
:101D10008008D8B0A5EF0EF0800E185C556E5650B6
:101D2000555CD8B0A5EF0EF05750555CD8B0A5EF74
:101D30000EF02652D8A4A1EF0EF05550142655509F
:101D4000152655500C2655500D26800E185CD8B01F
:101D5000C7EF0EF018508008556E0C50555CD8B087
:101D6000C7EF0EF00D50555CD8B0C7EF0EF02652FD
:101D7000D8A4C1EF0EF05550145C146E5550155C8C
:101D8000156E55500C5C0C6E55500D5C0D6E1200AE
:101D9000D3EC1EF039500208D8B4D1EF0EF007ECA6
:101DA0000FF039500108D8B406EF0FF0CDEC1EF05B
:101DB000B8EC1EF0145048EC0FF0200EEDEC1EF0C5
:101DC000200EEDEC1EF0ACEC1EF0155048EC0FF0C0
:101DD0001452D8A4FBEF0EF0CDEC1EF0B8EC1EF0C0
:101DE000200EEDEC1EF0BEEC1EF0200EEDEC1EF011
:101DF000200EEDEC1EF01552D8A406EF0FF0ACEC5F
:101E00001EF0200EEDEC1EF0BEEC1EF0120016507F
:101E10000108D8A40FEF0FF03150DFEC0FF016508F
:101E20000208D8A417EF0FF03250DFEC0FF0165075
:101E30000308D8A41FEF0FF03350DFEC0FF016505B
:101E40000408D8A427EF0FF03450DFEC0FF0165041
:101E50000508D8A42FEF0FF03550DFEC0FF0165027
:101E60000608D8A437EF0FF03650DFEC0FF016500D
:101E70000708D8A43FEF0FF03750DFEC0FF01650F3
:101E80000808D8A447EF0FF03850DFEC0FF012002D
:101E9000536EC00E535CD8B08FEF0FF05350000854
:101EA000D8B08FEF0FF02D0EEDEC1EF05350C008A0
:101EB0005A6E010E5B6ED3EC1FF0556E55505B6E83
:101EC0000A0E5C6EF3EC1FF0546E5450300FEDECC4
:101ED0001EF05350C0085A6E010E5B6ED3EC1FF01B
:101EE000576E5750586E0A0E596EE2EC1FF0566E40
:101EF0005650300FEDEC1EF02E0EEDEC1EF0535050
:101F0000010B0108D8A48AEF0FF0350EEDEC1EF09E
:101F10008DEF0FF0300EEDEC1EF0DEEF0FF0C00E87
:101F2000535CD8A0DEEF0FF053500008D8B0DEEFBE
:101F30000FF053500001C008D8A4A4EF0FF0200EFA
:101F4000EDEC1EF0A7EF0FF02B0EEDEC1EF0C00E27
:101F5000535C5A6E010E5B6ED3EC1FF0556E5550FC
:101F60005B6E0A0E5C6EF3EC1FF0546E5450300F33
:101F7000EDEC1EF0C00E535C5A6E010E5B6ED3EC9E
:101F80001FF0576E5750586E0A0E596EE2EC1FF054
:101F9000566E5650300FEDEC1EF02E0EEDEC1EF08E
:101FA0005350010B0108D8A4DBEF0FF0350EEDEC18
:101FB0001EF0DEEF0FF0300EEDEC1EF01200516E51
:101FC00051500108D8A4E7EF0FF07EEC1BF0515000
:101FD0000208D8A4EEEF0FF079EC1BF05150030883
:101FE000D8A4F5EF0FF0B1EC1BF051500408D8A4C1
:101FF000FCEF0FF0ACEC1BF051500508D8A403EF38
:1020000010F09FEC1AF051500608D8A40AEF10F017
:102010009AEC1AF051500708D8A411EF10F05FECB9
:102020001BF051500808D8A418EF10F05AEC1BF020
:1020300051500908D8A41FEF10F02EEC1BF051509E
:102040000A08D8A426EF10F029EC1BF051500B0819
:10205000D8A42DEF10F08CEC1BF051500C08D8A434
:1020600034EF10F087EC1BF051500D08D8A43BEF73
:1020700010F09DEC1BF051500E08D8A442EF10F068
:1020800098EC1BF051500F08D8A449EF10F04EEC1B
:102090001BF051501008D8A450EF10F049EC1BF081
:1020A00051501108D8A457EF10F06DEC1BF05150AF
:1020B0001208D8A45EEF10F068EC1BF05150130822
:1020C000D8A465EF10F01AEC1BF051501408D8A4F6
:1020D0006CEF10F015EC1BF051501508D8A473EFFD
:1020E00010F00FEC1BF051501608D8A47AEF10F046
:1020F0000AEC1BF051501708D8A481EF10F001EC46
:102100001BF051501808D8A488EF10F0FCEC1AF01E
:1021100051501908D8A48FEF10F0EDEC1AF051507F
:102120001A08D8A496EF10F0E8EC1AF051501B08EA
:10213000D8A49DEF10F0DFEC1AF051501C08D8A481
:10214000A4EF10F0DAEC1AF051501D08D8A4ABEF50
:1021500010F0D1EC1AF051501E08D8A4B2EF10F0D4
:10216000CCEC1AF051501F08D8A4B9EF10F0C6EC0F
:102170001AF051502008D8A4C0EF10F0C1EC1AF0AA
:1021800051502108D8A4C7EF10F0B8EC1AF0515004
:102190002208D8A4CEEF10F0B3EC1AF05150230867
:1021A000D8A4D5EF10F0ADEC1AF051502408D8A403
:1021B000DCEF10F0A8EC1AF01200D3EC1EF024ECC7
:1021C0001DF0CAEC1EF0A6EC1EF00C50145CD8A05A
:1021D000EFEF10F00D50155CD8B002EF11F00C507D
:1021E000145CD8B0F5EF10F0142A0D50155CD8B07F
:1021F000FBEF10F0152A31EC11F0275031EC1FF0F5
:10220000E5EF10F01200D3EC1EF024EC1DF0CAEC48
:102210001EF076EC1EF015500D6E14500C6E14501E
:102220000008D8A019EF11F015500008D8B030EF11
:1022300011F014500008D8B021EF11F0010E145C19
:10224000146E15500008D8B029EF11F0010E155C7E
:10225000156E31EC11F0275031EC1FF00FEF11F03B
:1022600012001550536E1450E3EF15F0536EB1EC9D
:1022700011F02852D8A47DEF11F053500108D8A4D2
:1022800045EF11F00480B7EC1FF053500208D8A4BA
:102290004DEF11F00482B5EC1FF053500308D8A4A1
:1022A00055EF11F00484B3EC1FF053500408D8A488
:1022B0005DEF11F00486B1EC1FF053500508D8A46F
:1022C00065EF11F00488AFEC1FF053500608D8A456
:1022D0006DEF11F0048AADEC1FF053500708D8A43D
:1022E00075EF11F0048CABEC1FF053500808D8A424
:1022F0007DEF11F0048EA9EC1FF028500108D8A43E
:10230000AEEF11F053500108D8A48DEF11F0048006
:10231000B7EC1FF00488AFEC1FF053500208D8A4AC
:1023200098EF11F00482B5EC1FF0048AADEC1FF0B9
:1023300053500308D8A4A3EF11F00484B3EC1FF0AA
:10234000048CABEC1FF053500408D8A4AEEF11F08E
:102350000486B1EC1FF0048EA9EC1FF05350166EEA
:1023600012000490B7EC1FF00492B5EC1FF0049437
:10237000B3EC1FF00496B1EC1FF00498AFEC1FF023
:10238000049AADEC1FF0049CABEC1FF0049EA9EF87
:102390001FF02FEC17F05250076E5350086E00924A
:1023A00000BC0082009400BE008423500108D8A421
:1023B0007BEF12F000A47BEF12F0096A0A6A075063
:1023C000215CD8A4EBEF11F00850225CD8A4EBEF0D
:1023D00011F00C0E096E07501D5CD8A4F7EF11F038
:1023E00008501E5CD8A4F7EF11F0020E096E0750DA
:1023F0001F5CD8A403EF12F00850205CD8A403EFB0
:1024000012F0010E096E0750195CD8A40FEF12F0FC
:1024100008501A5CD8A40FEF12F0040E096E075092
:102420001B5CD8A41BEF12F008501C5CD8A41BEF57
:1024300012F0080E096E07503B5CD8A427EF12F08B
:1024400008503C5CD8A427EF12F0010E0A6E07502A
:102450003D5CD8A433EF12F008503E5CD8A433EFB3
:1024600012F0020E0A6E07503F5CD8A43FEF12F044
:102470000850405CD8A43FEF12F0040E0A6E0750DB
:10248000415CD8A44BEF12F00850425CD8A44BEF4B
:1024900012F0080E0A6E0750435CD8A457EF12F0F2
:1024A0000850445CD8A457EF12F0100E0A6E075083
:1024B000455CD8A463EF12F00850465CD8A463EFE3
:1024C00012F0200E0A6E0750475CD8A46FEF12F08E
:1024D0000850485CD8A46FEF12F0400E0A6E075007
:1024E000495CD8A47BEF12F008504A5CD8A47BEF7B
:1024F00012F0800E0A6E1200096A82AE81EF12F0AD
:10250000092A82AC86EF12F0020E092682AA8BEF0E
:1025100012F0040E092682A890EF12F0080E092688
:102520000A6A82A095EF12F00A2A82A29AEF12F0AC
:10253000020E0A2682A49FEF12F0040E0A2682A63B
:10254000A4EF12F0080E0A2683A0A9EF12F0100ED5
:102550000A2683A2AEEF12F0200E0A2683A4B3EF60
:1025600012F0400E0A2683A6B8EF12F0800E0A265B
:102570001200146A156A010E166EFF0E176E800E99
:10258000186E100E196E100E1A6E100E1B6E110EB4
:102590001C6E120E1D6E2F0E1E6E120E1F6E350E4D
:1025A000206E100E216E0D0E226E010E236E020E95
:1025B000246E020E256E010E266E0F0E276E286AFF
:1025C000800E296E800E2A6E800E2B6E800E2C6E71
:1025D000800E2D6E800E2E6E800E2F6E800E306E51
:1025E000030E316E0D0E326E070E336E0F0E346E0B
:1025F000090E356E050E366E110E376E0B0E386EE7
:10260000396A040E3A6E100E3B6E010E3C6E100ECF
:102610003D6E020E3E6E100E3F6E030E406E100EAB
:10262000416E040E426E100E436E050E446E100E87
:10263000456E060E466E100E476E070E486E100E63
:10264000496E080E4A6E4B6A4C6A4D6A1200010EC2
:10265000506E14507DEC1FF0020E506E15507DEC44
:102660001FF0030E506E16507DEC1FF0050E506EDD
:1026700018507DEF1FF0506A2A0E7DEC1FF0010EFE
:10268000506E14507DEC1FF0020E506E15507DEC14
:102690001FF0030E506E16507DEC1FF0040E506EAE
:1026A00017507DEC1FF0050E506E18507DEC1FF09A
:1026B000060E506E19507DEC1FF0070E506E1A502A
:1026C0007DEC1FF0080E506E1B507DEC1FF0090EC4
:1026D000506E1C507DEC1FF00A0E506E1D507DECAC
:1026E0001FF00B0E506E1E507DEC1FF00C0E506E46
:1026F0001F507DEC1FF00D0E506E20507DEC1FF032
:102700000E0E506E21507DEC1FF00F0E506E2250B9
:102710007DEC1FF0100E506E23507DEC1FF0110E5B
:10272000506E24507DEC1FF0120E506E25507DEC43
:102730001FF0130E506E26507DEC1FF0140E506EDD
:1027400027507DEC1FF0150E506E28507DEC1FF0C9
:10275000160E506E29507DEC1FF0170E506E2A5049
:102760007DEC1FF0180E506E2B507DEC1FF0190EF3
:10277000506E2C507DEC1FF01A0E506E2D507DECDB
:102780001FF01B0E506E2E507DEC1FF01C0E506E75
:102790002F507DEC1FF01D0E506E30507DEC1FF061
:1027A0001E0E506E31507DEC1FF01F0E506E3250D9
:1027B0007DEC1FF0200E506E33507DEC1FF0210E8B
:1027C000506E34507DEC1FF0220E506E35507DEC73
:1027D0001FF0230E506E36507DEC1FF0240E506E0D
:1027E00037507DEC1FF0250E506E38507DEC1FF0F9
:1027F000260E506E39507DEC1FF0270E506E3A5069
:102800007DEC1FF0280E506E3B507DEC1FF0290E22
:10281000506E3C507DEC1FF02A0E506E3D507DEC0A
:102820001FF02B0E506E3E507DEC1FF02C0E506EA4
:102830003F507DEC1FF02D0E506E40507DEC1FF090
:102840002E0E506E41507DEC1FF02F0E506E4250F8
:102850007DEC1FF0300E506E43507DEC1FF0310EBA
:10286000506E44507DEC1FF0320E506E45507DECA2
:102870001FF0330E506E46507DEC1FF0340E506E3C
:1028800047507DEC1FF0350E506E48507DEC1FF028
:10289000360E506E49507DEC1FF0370E506E4A5088
:1028A0007DEC1FF0380E506E4B507DEC1FF0390E52
:1028B000506E4C507DEC1FF03A0E506E4D507DEF37
:1028C0001FF0010E506E92EC1FF05150146E020E6C
:1028D000506E92EC1FF05150156E030E506E92EC3C
:1028E0001FF05150166E040E506E92EC1FF05150B6
:1028F000176E050E506E92EC1FF05150186E060EBA
:10290000506E92EC1FF05150196E070E506E92EC03
:102910001FF051501A6E080E506E92EC1FF051507D
:102920001B6E090E506E92EC1FF051501C6E0A0E79
:10293000506E92EC1FF051501D6E0B0E506E92ECCB
:102940001FF051501E6E0C0E506E92EC1FF0515045
:102950001F6E0D0E506E92EC1FF05150206E0E0E39
:10296000506E92EC1FF05150216E0F0E506E92EC93
:102970001FF05150226E100E506E92EC1FF051500D
:10298000236E110E506E92EC1FF05150246E120EF9
:10299000506E92EC1FF05150256E130E506E92EC5B
:1029A0001FF05150266E140E506E92EC1FF05150D5
:1029B000276E150E506E92EC1FF05150286E160EB9
:1029C000506E92EC1FF05150296E170E506E92EC23
:1029D0001FF051502A6E180E506E92EC1FF051509D
:1029E0002B6E190E506E92EC1FF051502C6E1A0E79
:1029F000506E92EC1FF051502D6E1B0E506E92ECEB
:102A00001FF051502E6E1C0E506E92EC1FF0515064
:102A10002F6E1D0E506E92EC1FF05150306E1E0E38
:102A2000506E92EC1FF05150316E1F0E506E92ECB2
:102A30001FF05150326E200E506E92EC1FF051502C
:102A4000336E210E506E92EC1FF05150346E220EF8
:102A5000506E92EC1FF05150356E230E506E92EC7A
:102A60001FF05150366E240E506E92EC1FF05150F4
:102A7000376E250E506E92EC1FF05150386E260EB8
:102A8000506E92EC1FF05150396E270E506E92EC42
:102A90001FF051503A6E280E506E92EC1FF05150BC
:102AA0003B6E290E506E92EC1FF051503C6E2A0E78
:102AB000506E92EC1FF051503D6E2B0E506E92EC0A
:102AC0001FF051503E6E2C0E506E92EC1FF0515084
:102AD0003F6E2D0E506E92EC1FF05150406E2E0E38
:102AE000506E92EC1FF05150416E2F0E506E92ECD2
:102AF0001FF05150426E300E506E92EC1FF051504C
:102B0000436E310E506E92EC1FF05150446E320EF7
:102B1000506E92EC1FF05150456E330E506E92EC99
:102B20001FF05150466E340E506E92EC1FF0515013
:102B3000476E350E506E92EC1FF05150486E360EB7
:102B4000506E92EC1FF05150496E370E506E92EC61
:102B50001FF051504A6E380E506E92EC1FF05150DB
:102B60004B6E390E506E92EC1FF051504C6E3A0E77
:102B7000506E92EC1FF051504D6E1450175CD8B04F
:102B8000C4EF15F01750146E1550175CD8B0CBEF8A
:102B900015F01750156E1200526E5250536E53526C
:102BA000D8B4E2EF15F006929DEC1FF0010E21EC77
:102BB0001FF006829DEC1FF0010E21EC1FF0530662
:102BC000CFEF15F01200546E059EA1EC1FF0040E1D
:102BD000556E5350800B0008D8B0F4EF15F0058CFB
:102BE000A3EC1FF0F7EF15F0059CA3EC1FF0058A8E
:102BF000A5EC1FF0059AA5EC1FF05350400B000800
:102C0000D8B008EF16F0058CA3EC1FF00BEF16F010
:102C1000059CA3EC1FF0058AA5EC1FF0059AA5EC16
:102C20001FF05350200B0008D8B01CEF16F0058C95
:102C3000A3EC1FF01FEF16F0059CA3EC1FF0058A14
:102C4000A5EC1FF0059AA5EC1FF05350100B0008DF
:102C5000D8B030EF16F0058CA3EC1FF033EF16F070
:102C6000059CA3EC1FF0058AA5EC1FF0059AA5ECC6
:102C70001FF05350080B0008D8B044EF16F0058C35
:102C8000A3EC1FF047EF16F0059CA3EC1FF0058A9C
:102C9000A5EC1FF0059AA5EC1FF05350040B00089B
:102CA000D8B058EF16F0058CA3EC1FF05BEF16F0D0
:102CB000059CA3EC1FF0058AA5EC1FF0059AA5EC76
:102CC0001FF05350020B0008D8B06CEF16F0058CC3
:102CD000A3EC1FF06FEF16F0059CA3EC1FF0058A24
:102CE000A5EC1FF0059AA5EC1FF05350010B00084E
:102CF000D8B080EF16F0058CA3EC1FF083EF16F030
:102D0000059CA3EC1FF0058AA5EC1FF0059AA5EC25
:102D10001FF05450800B0008D8B094EF16F0058CCB
:102D2000A3EC1FF097EF16F0059CA3EC1FF0058AAB
:102D3000A5EC1FF0059AA5EC1FF05450400B0008BD
:102D4000D8B0A8EF16F0058CA3EC1FF0ABEF16F08F
:102D5000059CA3EC1FF0058AA5EC1FF0059AA5ECD5
:102D60001FF05450200B0008D8B0BCEF16F0058CB3
:102D7000A3EC1FF0BFEF16F0059CA3EC1FF0058A33
:102D8000A5EC1FF0059AA5EC1FF05450100B00089D
:102D9000D8B0D0EF16F0058CA3EC1FF0D3EF16F0EF
:102DA000059CA3EC1FF0058AA5EC1FF0059AA5EC85
:102DB0001FF05450080B0008D8B0E4EF16F0058C53
:102DC000A3EC1FF0E7EF16F0059CA3EC1FF0058ABB
:102DD000A5EC1FF0059AA5EC1FF05450040B000859
:102DE000D8B0F8EF16F0058CA3EC1FF0FBEF16F04F
:102DF000059CA3EC1FF0058AA5EC1FF0059AA5EC35
:102E00001FF05450020B0008D8B00CEF17F0058CDF
:102E1000A3EC1FF00FEF17F0059CA3EC1FF0058A41
:102E2000A5EC1FF0059AA5EC1FF05450010B00080B
:102E3000D8B020EF17F0058CA3EC1FF023EF17F0AC
:102E4000059CA3EC1FF0058AA5EC1FF0059AA5ECE4
:102E50001FF0552EE9EF15F0058EA1EF1FF0526A15
:102E6000536A009CFF0E546EFF0E556E008E0D0EC1
:102E7000566E1A0E576E0190019254500008D8B049
:102E800043EF17F084A44DEF17F0010E39EC1FF05B
:102E9000010E545C546E3DEF17F05452D8A454EF19
:102EA00017F0009EA9EF19F0060E29EC1FF0FF0E97
:102EB000556E55500008D8B05FEF17F084A478EF36
:102EC00017F0FF0E546E54500008D8B069EF17F099
:102ED00084A473EF17F0020E6DEC1FF0010E545C2A
:102EE000546E63EF17F0010E555C556E59EF17F0F5
:102EF0005552D8A47FEF17F0009EA9EF19F0019466
:102F000001B00184AAEC19F05850546E019001B43C
:102F100001805650545CD8B09CEF17F0008E0182AF
:102F2000019401B00184AAEC19F05850546E01903C
:102F300001B401809EEF17F0009E0192019401B050
:102F40000184AAEC19F05850546E019001B401802C
:102F50005650545CD8B0BCEF17F0009C01B2008C06
:102F6000019401B00184AAEC19F05850546E0190FC
:102F700001B40180BFEF17F0009C01A2008C019208
:102F800000BC0182019401B00184AAEC19F05850F0
:102F9000546E019001B401805650545CD8B0E2EFF9
:102FA00017F001A2D6EF17F0100E5226019401B0CF
:102FB0000184AAEC19F05850546E019001B40180BC
:102FC000EEEF17F001B2E7EF17F0100E522601B244
:102FD000EDEF17F00182EEEF17F00192019401B0CE
:102FE0000184AAEC19F05850546E019001B401808C
:102FF0005650545CD8B00EEF18F001A202EF18F052
:10300000080E5226019401B00184AAEC19F0585020
:10301000546E019001B401801AEF18F001B213EF61
:1030200018F0080E522601B219EF18F001821AEFBB
:1030300018F00192019401B00184AAEC19F05850E3
:10304000546E019001B401805650545CD8B03AEFF0
:1030500018F001A22EEF18F0040E5226019401B0D0
:103060000184AAEC19F05850546E019001B401800B
:1030700046EF18F001B23FEF18F0040E522601B2ED
:1030800045EF18F0018246EF18F00192019401B06B
:103090000184AAEC19F05850546E019001B40180DB
:1030A0005650545CD8B066EF18F001A25AEF18F0F1
:1030B000020E5226019401B00184AAEC19F0585076
:1030C000546E019001B4018072EF18F001B26BEF01
:1030D00018F0020E522601B271EF18F0018272EF61
:1030E00018F00192019401B00184AAEC19F0585033
:1030F000546E019001B401805650545CD8B091EFE9
:1031000018F001A285EF18F0522A019401B0018451
:10311000AAEC19F05850546E019001B401809CEF54
:1031200018F001B295EF18F0522A01B29BEF18F097
:1031300001829CEF18F00192019401B00184AAEC85
:1031400019F05850546E019001B401805650545CEF
:10315000D8B0BCEF18F001A2B0EF18F0200E532643
:10316000019401B00184AAEC19F05850546E0190FA
:1031700001B40180C8EF18F001B2C1EF18F0200EC1
:10318000532601B2C7EF18F00182C8EF18F0019280
:10319000019401B00184AAEC19F05850546E0190CA
:1031A00001B401805650545CD8B0E8EF18F001A289
:1031B000DCEF18F0100E5326019401B00184AAEC44
:1031C00019F05850546E019001B40180F4EF18F0DA
:1031D00001B2EDEF18F0100E532601B2F3EF18F024
:1031E0000182F4EF18F00192019401B00184AAEC7D
:1031F00019F05850546E019001B401805650545C3F
:10320000D8B014EF19F001A208EF19F0080E5326F8
:10321000019401B00184AAEC19F05850546E019049
:1032200001B4018020EF19F001B219EF19F0080E76
:10323000532601B21FEF19F0018220EF19F001921D
:10324000019401B00184AAEC19F05850546E019019
:1032500001B401805650545CD8B040EF19F001A27F
:1032600034EF19F0040E5326019401B00184AAEC46
:1032700019F05850546E019001B401804CEF19F0D0
:1032800001B245EF19F0040E532601B24BEF19F0CD
:1032900001824CEF19F00192019401B00184AAEC73
:1032A00019F05850546E019001B401805650545C8E
:1032B000D8B06CEF19F001A260EF19F0020E53269E
:1032C000019401B00184AAEC19F05850546E019099
:1032D00001B4018078EF19F001B271EF19F0020E1C
:1032E000532601B277EF19F0018278EF19F00192BD
:1032F000019401B00184AAEC19F05850546E019069
:1033000001B401805650545CD8B097EF19F001A277
:103310008BEF19F0532A019401B00184AAEC19F043
:103320005850546E019001B40180A2EF19F001B21F
:103330009BEF19F0532A01B2A1EF19F00182A2EF1D
:1033400019F0019201A0A9EF19F0009E009C536AA8
:10335000526A1200586A019684B4018684A4B6EFBA
:1033600019F001A6BCEF19F0B9EF19F001B6BCEFE6
:1033700019F01E0E585CD8B0C4EF19F0010E41ECE4
:103380001FF0582AAEEF19F058501E08D8A4CAEF03
:1033900019F001841200550EEDEC1EF0730EEDECE9
:1033A0001EF0650EEDEC1EF0200EEDEC1EF0610E31
:1033B000EDEC1EF0630EEDEC1EF0740EEDEC1EF065
:1033C000200EEDEC1EF0610EEDEC1EF0730EEDEC38
:1033D0001EF0200EEDEC1EF0500EEDEC1EF0720E05
:1033E000EDEC1EF0730EEDEC1EF0650EEDEC1EF034
:1033F000740EEDEF1EF013EC1AF0CAEC1EF010EF95
:103400001CF0500EEDEC1EF0720EEDEC1EF0650E91
:10341000EDEC1EF0730EEDEC1EF0650EEDEC1EF003
:10342000740EEDEF1EF0500EEDEC1EF06F0EEDEC95
:103430001EF0770EEDEC1EF0650EEDEC1EF0720E38
:10344000EDEC1EF0750EEDEC1EF0700EEDEF1EF0C3
:103450004D0EEDEC1EF0610EEDEC1EF0780EEDEC75
:103460001EF0200EEDEC1EF0560EEDEC1EF06F0E71
:10347000EDEC1EF06C0EEDEC1EF0750EEDEC1EF09A
:103480006D0EEDEC1EF0650EEDEC1EF03A0EEDEF5C
:103490001EF0560EEDEC1EF06F0EEDEC1EF06C0EF5
:1034A000EDEC1EF0750EEDEC1EF06D0EEDEC1EF069
:1034B000650EEDEC1EF0200EEDEC1EF04F0EEDEC67
:1034C0001EF06E0EEDEC1EF06C0EEDEC1EF0790EA3
:1034D000EDEF1EF0490EEDEC1EF06E0EEDEC1EF061
:1034E000700EEDEC1EF0750EEDEC1EF0740EEDECB2
:1034F0001EF0200EEDEC1EF04F0EEDEC1EF06E0EE9
:10350000EDEC1EF06C0EEDEC1EF0790EEDEF1EF002
:103510004E0EEDEC1EF06F0EEDEC1EF0720EEDECAB
:103520001EF06D0EEDEC1EF0610EEDEC1EF06C0E5B
:10353000EDEF1EF09FEC1AF0320EEDEF1EF0440E90
:10354000EDEC1EF0410EEDEC1EF0430EEDEF1EF023
:10355000ADEC1AF0320EEDEF1EF0500EEDEC1EF059
:10356000430EEDEF1EF0B8EC1AF0320EEDEF1EF048
:10357000440EEDEC1EF0410EEDEC1EF0540EEDEF9E
:103580001EF0C6EC1AF0320EEDEF1EF04D0EEDEC13
:103590001EF0440EEDEF1EF0D1EC1AF0320EEDEFFE
:1035A0001EF0440EEDEC1EF0430EEDEC1EF0430E4B
:1035B000EDEF1EF0DFEC1AF0320EEDEF1EF0530EC1
:1035C000EDEC1EF0410EEDEC1EF0540EEDEF1EF092
:1035D000EDEC1AF0320EEDEF1EF0560EEDEC1EF093
:1035E000690EEDEC1EF0640EEDEC1EF0650EEDECD8
:1035F0001EF06F0EEDEF1EF001EC1BF0320EEDEF42
:103600001EF0560EEDEC1EF0430EEDEC1EF0520EC9
:10361000EDEF1EF00FEC1BF0320EEDEF1EF0540E2E
:10362000EDEC1EF0560EEDEF1EF01AEC1BF0320E14
:10363000EDEF1EF0540EEDEC1EF0750EEDEC1EF0ED
:103640006E0EEDEC1EF0650EEDEC1EF0720EEDEF61
:103650001EF02EEC1BF0320EEDEF1EF0440EEDECE2
:103660001EF0560EEDEC1EF0440EEDEC1EF02D0E8D
:10367000EDEC1EF0410EEDEC1EF0750EEDEC1EF0C3
:10368000640EEDEC1EF0690EEDEC1EF06F0EEDEF2A
:103690001EF04EEC1BF0320EEDEF1EF0530EEDEC73
:1036A0001EF0410EEDEC1EF0430EEDEC1EF0440E4C
:1036B000EDEF1EF05FEC1BF0320EEDEF1EF0440E4E
:1036C000EDEC1EF0560EEDEC1EF0440EEDEF1EF08C
:1036D0006DEC1BF0320EEDEF1EF0540EEDEC1EF013
:1036E000610EEDEC1EF0700EEDEC1EF0650EEDEFD0
:1036F0001EF07EEC1BF0320EEDEF1EF0410EEDECF5
:103700001EF0750EEDEC1EF0780EEDEF1EF08CEC59
:103710001BF0320EEDEF1EF04C0EEDEC1EF0690EBC
:10372000EDEC1EF06E0EEDEC1EF0650EEDEF1EF0F2
:103730009DEC1BF0320EEDEF1EF0500EEDEC1EF086
:10374000680EEDEC1EF06F0EEDEC1EF06E0EEDEC63
:103750001EF06F0EEDEF1EF0B1EC1BF0320EEDEF30
:103760001EF0430EEDEC1EF0440EEDEF1EF0D0EC1B
:103770001EF001EC1CF03A0EEDEC1EF0200EEDEC0C
:103780001EF0440EEDEC1EF06F0EEDEC1EF0750E0B
:10379000EDEC1EF0620EEDEC1EF06C0EEDEC1EF08A
:1037A000650EEDEC1EF0200EEDEC1EF0200EEDECA3
:1037B0001EF0200EEDEF1EF0D0EC1EF001EC1CF020
:1037C0003A0EEDEC1EF0200EEDEC1EF0530EEDEC7B
:1037D0001EF0690EEDEC1EF06E0EEDEC1EF0670EA5
:1037E000EDEC1EF06C0EEDEC1EF0650EEDEC1EF037
:1037F000200EEDEC1EF0200EEDEC1EF0200EEDEF95
:103800001EF0490EEDEC1EF06E0EEDEC1EF0700E8B
:10381000EDEC1EF0750EEDEC1EF0740EEDEF1EF0EB
:10382000560EEDEC1EF06F0EEDEC1EF06C0EEDEC96
:103830001EF0750EEDEC1EF06D0EEDEC1EF0650E3B
:10384000EDEF1EF0CDEC1EF0B8EC1EF030EF1DF0E9
:10385000CDEC1EF0B8EC1EF030EC1DF0200EEDECBF
:103860001EF0200EEDEC1EF0ACEC1EF04E0EEDEC5A
:103870001EF0650EEDEC1EF0780EEDEC1EF0740EF1
:10388000EDEF1EF0CDEC1EF0B8EC1EF030EC1DF0AC
:10389000200EEDEC1EF0200EEDEC1EF0ACEC1EF058
:1038A0002D0EEDEC1EF03E0EEDEF1EF0516E6EECA7
:1038B0001CF0200EEDEC1EF0430EEDEC1EF0680E39
:1038C000EDEC1EF05150300FEDEC1EF03A0EEDEF26
:1038D0001EF07AEC1CF0730EEDEF1EF04F0EEDECC7
:1038E0001EF0660EEDEC1EF0660EEDEC1EF0730E93
:1038F000EDEF1EF04F0EEDEC1EF0660EEDEC1EF03F
:10390000660EEDEC1EF0730EEDEC1EF0650EEDECA8
:103910001EF0740EEDEF1EF0490EEDEC1EF06E0E73
:10392000EDEC1EF0700EEDEC1EF0750EEDEC1EF0E1
:10393000740EEDEC1EF02D0EEDEC1EF0540EEDECC1
:103940001EF0790EEDEC1EF0700EEDEC1EF0650E23
:10395000EDEF1EF0520EEDEC1EF0650EEDEC1EF0DC
:10396000730EEDEC1EF0740EEDEC1EF06F0EEDEC30
:103970001EF0720EEDEC1EF0650EEDEC1EF0CAECC2
:103980001EF0440EEDEC1EF0650EEDEC1EF0660E22
:10399000EDEC1EF0610EEDEC1EF0750EEDEC1EF080
:1039A0006C0EEDEC1EF0740EEDEC1EF0730EEDEFF0
:1039B0001EF0520EEDEC1EF0650EEDEC1EF06C0EDE
:1039C000EDEC1EF0610EEDEC1EF0790EEDEC1EF04C
:1039D0002D0EEDEC1EF0540EEDEC1EF0650EEDEC30
:1039E0001EF0730EEDEC1EF0740EEDEF1EF024EFE2
:1039F0001DF024EC1DF0640EEDEC1EF0650EEDECF8
:103A00001EF06C0EEDEC1EF0610EEDEC1EF0790E6A
:103A1000EDEC1EF03A0EEDEC1EF0200EEDEF1EF078
:103A2000550EEDEC1EF0730EEDEC1EF0650EEDEC98
:103A30001EF0200EEDEC1EF024EC1DF03A0EEDEC25
:103A40001EF0200EEDEF1EF0520EEDEC1EF0610E9A
:103A5000EDEC1EF06D0EEDEC1EF0700EEDEF1EF0B5
:103A6000450EEDEC1EF0780EEDEC1EF0690EEDEC5F
:103A70001EF0740EEDEF1EF0480EEDEC1EF0610E20
:103A8000EDEC1EF0720EEDEC1EF0640EEDEC1EF08F
:103A9000770EEDEC1EF0610EEDEC1EF0720EEDEC0B
:103AA0001EF0650EEDEC1EF0200EEDEC1EF0530E38
:103AB000EDEC1EF0650EEDEC1EF0740EEDEC1EF05C
:103AC000750EEDEC1EF0700EEDEF1EF02BEC1EF0FF
:103AD0006E0EEDEC1EF0610EEDEC1EF06D0EEDECD9
:103AE0001EF0650EEDEC1EF0730EEDEF1EF04D0EA8
:103AF000EDEC1EF0610EEDEC1EF0780EEDEC1EF01C
:103B0000690EEDEC1EF06D0EEDEC1EF0750EEDEC99
:103B10001EF06D0EEDEC1EF0200EEDEC1EF0560EBC
:103B2000EDEC1EF06F0EEDEC1EF06C0EEDEC1EF0E9
:103B3000750EEDEC1EF06D0EEDEC1EF0650EEDEF6A
:103B40001EF0520EEDEC1EF0430EEDEC1EF0350EA5
:103B5000EDEC1EF0CAEC1EF0490EEDEC1EF0520E1C
:103B6000EDEC1EF02D0EEDEC1EF0540EEDEC1EF003
:103B7000650EEDEC1EF0730EEDEC1EF0740EEDEF25
:103B80001EF0520EEDEC1EF0430EEDEC1EF0350E65
:103B9000EDEC1EF0CAEC1EF0490EEDEC1EF0520EDC
:103BA000EDEC1EF02D0EEDEC1EF0F5EF1DF0E3EC4C
:103BB0001DF0CAEC1EF0F5EF1DF0ECEC1DF0CAECA8
:103BC0001EF0F5EF1DF04C0EEDEC1EF0430EEDEC8B
:103BD0001EF0440EEDEF1EF04C0EEDEC1EF0450E07
:103BE000EDEC1EF0440EEDEF1EF0530EEDEC1EF06A
:103BF000650EEDEC1EF0740EEDEC1EF0750EEDECA6
:103C00001EF0700EEDEF1EF04E0EEDEC1EF06F0E7E
:103C1000EDEF1EF0590EEDEC1EF0650EEDEC1EF012
:103C2000730EEDEF1EF0640EEDEC1EF0420EEDEFA4
:103C30001EF0410EEDEC1EF06C0EEDEC1EF0770E5A
:103C4000EDEC1EF0610EEDEC1EF0790EEDEC1EF0C9
:103C5000730EEDEF1EF0430EEDEC1EF0680EEDEC72
:103C60001EF0610EEDEC1EF06E0EEDEC1EF06E0E11
:103C7000EDEC1EF0650EEDEC1EF06C0EEDEF1EF09F
:103C8000440EEDEC1EF0650EEDEC1EF06C0EEDEC4E
:103C90001EF0610EEDEC1EF0790EEDEF1EF0520EEF
:103CA000EDEC1EF0690EEDEC1EF0670EEDEC1EF073
:103CB000680EEDEC1EF0740EEDEF1EF04C0EEDEC08
:103CC0001EF0610EEDEC1EF0730EEDEC1EF0740EA6
:103CD000EDEF1EF04C0EEDEC1EF0650EEDEC1EF05F
:103CE000660EEDEC1EF0740EEDEF1EF0440EEDECE2
:103CF0001EF06F0EEDEC1EF0770EEDEC1EF06E0E6A
:103D0000EDEF1EF04F0EEDEC1EF0660EEDEC1EF02A
:103D1000660EEDEF1EF04F0EEDEC1EF06E0EEDEFA9
:103D20001EF0430EEDEC1EF0680EEDEF1EF06D0E72
:103D3000EDEC1EF0730EEDEF1EF02F0EEDEC1EF00D
:103D4000630EEDEC1EF03A0EEDEF1EF0550EEDECAD
:103D50001EF0700EEDEF1EF0520EEDEC1EF03A0E5E
:103D6000EDEF1EF0610EEDEC1EF03A0EEDEF1EF0E1
:103D70004C0EEDEC1EF03A0EEDEF1EF04D0EEDEC9C
:103D80001EF0750EEDEC1EF0740EEDEC1EF0650EDF
:103D9000EDEF1EF0200EEDEF1EF0A80EF8EF1EF076
:103DA000800EF8EF1EF0080EF8EC1EF0010EF8EC95
:103DB0001EF0C80E5FEC1FF0020EF8EC1EF0C80EED
:103DC0005FEC1FF0060EF8EC1EF00C0EF8EC1EF087
:103DD000C80E5FEF1FF002505B6E5B6E0388BBEC9A
:103DE0001FF05B380F0B09EC1FF05B5009EF1FF061
:103DF000536E0398BBEC1FF053380F0B09EC1FF008
:103E0000820E5FEC1FF0535009EC1FF0820E5FEF43
:103E10001FF05C6E038AB9EC1FF05C50BDEC1FF024
:103E2000039AB9EC1FF0FA0E6DEF1FF0000EBDEC17
:103E30001FF00398BBEC1FF0039AB9EC1FF0926AD5
:103E40001200546E54505A6E640E5B6E0A0E49EFA7
:103E50001FF0586E58505A6E640E5B6E010E49EF9B
:103E60001FF0536E53505A6E0A0E5B6E010E49EFEF
:103E70001FF0586E58505A6E050E5B6E010E49EFDA
:103E80001FF0596E59505A6E010E5B6E010E49EFCC
:103E90001FF05C6EFF0E5D6E5B505F6E5A505E6E83
:103EA0003B0E5D24D8B051EF1FF05E2E50EF1FF097
:103EB0005F2E4EEF1FF05C2E4CEF1FF01200546E81
:103EC0005450556E5552D8B46CEF1FF00A0E6DEC7D
:103ED0001FF0550662EF1FF012005D6EFB0E5E6E66
:103EE000FE0E5F6E5D505E24D8A0000C5F2474EF60
:103EF0001FF01200070EC16E1200516E5050A96ED5
:103F00005150A86EA69EA69CA684F29E550EA76E42
:103F1000AA0EA76EA682F28EA6B28CEF1FF0A19811
:103F2000A6941200516E5050A96EA69EA69CF29EB9
:103F3000A680A850516EF28E1200C7EF1FF0C7EF97
:103F40001FF0CAEF1FF0CAEF1FF0CAEF1FF0CAEF51
:103F50001FF0CDEF1FF0CDEF1FF0CDEF1FF0CDEF35
:103F60001FF0CDEF1FF0CDEF1FF0CDEF1FF0CDEF25
:103F70001FF0D0EF1FF0D0EF1FF05D6E5D500F0B04
:103F80005E6E0350F00B5E10036ED0EF1FF0065014
:103F9000846E12000550836E12000450816E120070
:103FA0000350806E12005B6E5B500008D8B0E0EFEB
:103FB0001FF0D8905A32010E5B5C5B6ED4EF1FF09D
:103FC0005A501200596E5952D8B4F1EF1FF059509F
:103FD000585CD8A0F1EF1FF05950585C586EE7EFCD
:103FE0001FF0585012005C6E5D6A5C52D8B404EF4A
:103FF00020F05C505B5CD8A004EF20F05C505B5C70
:104000005B6E5D2AF9EF1FF05D501200040E026E28
:0240100012009C
:0200000400F00A
:020000040030CA
:0E00000000220C0E000180000FC00FE00F4028
:00000001FF
